:100000000BC018C017C016C015C014C055C012C010
:1000100011C010C00FC00EC011241FBECFEDCDBF48
:1000200010E0A0E6B0E001C01D92A836B107E1F7EC
:100030000BD115C1E5CF80916500882311F0D99AC5
:1000400001C0D99880916700882311F0DB9A089548
:10005000DB98089580916100882369F19091610097
:100060009130E9F480916600823228F410926200A7
:10007000109265000CC080916600853258F0809126
:100080006600823338F4909362009093650010927A
:10009000670010C080916600853360F004C08091D5
:1000A0006100823039F481E08093620080936500C2
:1000B00080936700C0DF08951F920F920FB60F92D2
:1000C00011242F933F934F935F936F937F938F935D
:1000D0009F93AF93BF93EF93FF938091600088232A
:1000E000C1F0CF9B0AC0809163009091640001969B
:1000F000909364008093630015C0809163008093A7
:100100006600109260001092640010926300A2DFFB
:1001100009C0CF9B07C081E080936000109264000B
:1001200010926300FF91EF91BF91AF919F918F91DA
:100130007F916F915F914F913F912F910F900FBEE3
:100140000F901F90189589B380780895682F20E04C
:1001500030E044EF51E089B38078861711F080E0F9
:100160000895842F952F0197F1F72F5F3F4F87E276
:100170002031380781F781E0089580E29EE428EC81
:1001800030E0E22FF32F3197F1F70197D1F789B3E0
:100190008078DCDF882311F481E0089582E00895FF
:1001A000D09AD19AD39AD49AD59ADF9AD898DC98D3
:1001B000DB98D998DD981092620010926500109239
:1001C000670083B7816083BF89B7826089BF7894F5
:1001D0000895D89ADD9A80E49CE90197F1F7DD98BB
:1001E000D8988CE494E028EC30E0E22FF32F31979C
:1001F000F1F70197D1F780916200882321F1D89A15
:1002000080E49CE90197F1F7D89880ED97E028EC1D
:1002100030E0E22FF32F3197F1F70197D1F780917A
:100220006200882381F0DC9A80E49CE90197F1F771
:10023000DC9888EB9BE028EC30E0E22FF32F31973D
:10024000F1F70197D1F70895ABDF97DF8093610055
:1002500001DF809162008823E1F3BBDFFACFF894DD
:02026000FFCFCE
:00000001FF
